 jabsysinfo

 Timestamp is ffffffff (Sun Feb  7 06:28:15 2106)

 Preferred load address is 10000000

 Start         Length     Name                   Class
 0001:00000000 00000e8aH .text$mn                CODE
 0002:00000000 00000080H .idata$5                DATA
 0002:00000080 00000004H .00cfg                  DATA
 0002:00000084 00000004H .CRT$XCA                DATA
 0002:00000088 00000004H .CRT$XCZ                DATA
 0002:0000008c 00000004H .CRT$XIA                DATA
 0002:00000090 00000004H .CRT$XIZ                DATA
 0002:00000094 00000004H .CRT$XPA                DATA
 0002:00000098 00000004H .CRT$XPZ                DATA
 0002:0000009c 00000004H .CRT$XTA                DATA
 0002:000000a0 00000008H .CRT$XTZ                DATA
 0002:000000a4 00000000H .gfids$y                DATA
 0002:000000a8 000001a0H .rdata                  DATA
 0002:00000248 000000dcH .rdata$r                DATA
 0002:00000324 00000004H .rdata$sxdata           DATA
 0002:00000328 000002acH .rdata$zzzdbg           DATA
 0002:000005d4 00000004H .rtc$IAA                DATA
 0002:000005d8 00000004H .rtc$IZZ                DATA
 0002:000005dc 00000004H .rtc$TAA                DATA
 0002:000005e0 00000008H .rtc$TZZ                DATA
 0002:000005e8 000000e8H .xdata$x                DATA
 0002:000006d0 00000084H .edata                  DATA
 0002:00000754 00000050H .idata$2                DATA
 0002:000007a4 00000014H .idata$3                DATA
 0002:000007b8 00000080H .idata$4                DATA
 0002:00000838 000002caH .idata$6                DATA
 0003:00000000 00000020H .data                   DATA
 0003:00000020 00000058H .data$r                 DATA
 0003:00000078 00000370H .bss                    DATA
 0004:00000000 00000120H .rsrc$01                DATA
 0004:00000120 00000618H .rsrc$02                DATA

  Address         Publics by Value              Rva+Base       Lib:Object

 0000:00000000       ___guard_longjmp_count     00000000     <absolute>
 0000:00000000       ___hybrid_code_map         00000000     <absolute>
 0000:00000000       ___dynamic_value_reloc_table 00000000     <absolute>
 0000:00000000       ___x64_code_ranges_to_entry_points 00000000     <absolute>
 0000:00000000       ___guard_eh_cont_count     00000000     <absolute>
 0000:00000000       ___guard_fids_count        00000000     <absolute>
 0000:00000000       ___guard_iat_table         00000000     <absolute>
 0000:00000000       ___guard_iat_count         00000000     <absolute>
 0000:00000000       ___arm64x_native_entrypoint 00000000     <absolute>
 0000:00000000       ___arm64x_extra_rfe_table  00000000     <absolute>
 0000:00000000       ___arm64x_extra_rfe_table_size 00000000     <absolute>
 0000:00000000       ___hybrid_auxiliary_iat    00000000     <absolute>
 0000:00000000       ___arm64x_redirection_metadata_count 00000000     <absolute>
 0000:00000000       ___guard_fids_table        00000000     <absolute>
 0000:00000000       ___guard_longjmp_table     00000000     <absolute>
 0000:00000000       ___volatile_metadata       00000000     <absolute>
 0000:00000000       ___enclave_config          00000000     <absolute>
 0000:00000000       ___arm64x_redirection_metadata 00000000     <absolute>
 0000:00000000       ___AbsoluteZero            00000000     <absolute>
 0000:00000000       ___hybrid_code_map_count   00000000     <absolute>
 0000:00000000       ___guard_eh_cont_table     00000000     <absolute>
 0000:00000000       ___x64_code_ranges_to_entry_points_count 00000000     <absolute>
 0000:00000001       ___safe_se_handler_count   00000001     <absolute>
 0000:00000100       ___guard_flags             00000100     <absolute>
 0000:00000000       ___ImageBase               10000000     <linker-defined>
 0001:00000000       ??0exception@std@@QAE@ABV01@@Z 10001000 f i AccessBridgeSysInfo.obj
 0001:00000029       ??0exception@std@@QAE@QBD@Z 10001029 f i AccessBridgeSysInfo.obj
 0001:0000005e       ??0runtime_error@std@@QAE@ABV01@@Z 1000105e f i AccessBridgeSysInfo.obj
 0001:00000076       ??0runtime_error@std@@QAE@PBD@Z 10001076 f i AccessBridgeSysInfo.obj
 0001:0000008e       ??1runtime_error@std@@UAE@XZ 1000108e f i AccessBridgeSysInfo.obj
 0001:0000009f       ??_Eexception@std@@UAEPAXI@Z 1000109f f i AccessBridgeSysInfo.obj
 0001:0000009f       ??_Gexception@std@@UAEPAXI@Z 1000109f f i AccessBridgeSysInfo.obj
 0001:0000009f       ??_Gruntime_error@std@@UAEPAXI@Z 1000109f f i AccessBridgeSysInfo.obj
 0001:0000009f       ??_Eruntime_error@std@@UAEPAXI@Z 1000109f f i AccessBridgeSysInfo.obj
 0001:000000c9       ?what@exception@std@@UBEPBDXZ 100010c9 f i AccessBridgeSysInfo.obj
 0001:000000d7       _DllMain@12                100010d7 f   AccessBridgeSysInfo.obj
 0001:000000dd       _Java_com_sun_java_accessibility_internal_AccessBridge_isSysWow@8 100010dd f   AccessBridgeSysInfo.obj
 0001:0000013e       ??3@YAXPAXI@Z              1000113e f   MSVCRT:delete_scalar_size.obj
 0001:0000014c       ??_Etype_info@@UAEPAXI@Z   1000114c f i MSVCRT:std_type_info_static.obj
 0001:0000014c       ??_Gtype_info@@UAEPAXI@Z   1000114c f i MSVCRT:std_type_info_static.obj
 0001:000004af       __DllMainCRTStartup@12     100014af f   MSVCRT:dll_dllmain.obj
 0001:000004d2       ??3@YAXPAX@Z               100014d2 f   MSVCRT:delete_scalar.obj
 0001:00000524       ___security_init_cookie    10001524 f   MSVCRT:gs_support.obj
 0001:0000056f       ?__scrt_initialize_type_info@@YAXXZ 1000156f f   MSVCRT:tncleanup.obj
 0001:0000057b       ?__scrt_uninitialize_type_info@@YAXXZ 1000157b f   MSVCRT:tncleanup.obj
 0001:00000587       ___local_stdio_printf_options 10001587 f i MSVCRT:default_local_stdio_options.obj
 0001:0000058d       ___local_stdio_scanf_options 1000158d f i MSVCRT:default_local_stdio_options.obj
 0001:00000593       ___scrt_initialize_default_local_stdio_options 10001593 f   MSVCRT:default_local_stdio_options.obj
 0001:000005f4       ___scrt_acquire_startup_lock 100015f4 f   MSVCRT:utility.obj
 0001:00000626       ___scrt_dllmain_after_initialize_c 10001626 f   MSVCRT:utility.obj
 0001:00000651       ___scrt_dllmain_before_initialize_c 10001651 f   MSVCRT:utility.obj
 0001:0000065f       ___scrt_dllmain_crt_thread_attach 1000165f f   MSVCRT:utility.obj
 0001:0000067e       ___scrt_dllmain_crt_thread_detach 1000167e f   MSVCRT:utility.obj
 0001:0000068b       ___scrt_dllmain_exception_filter 1000168b f   MSVCRT:utility.obj
 0001:000006bf       ___scrt_dllmain_uninitialize_c 100016bf f   MSVCRT:utility.obj
 0001:000006e2       ___scrt_dllmain_uninitialize_critical 100016e2 f   MSVCRT:utility.obj
 0001:000006ef       ___scrt_initialize_crt     100016ef f   MSVCRT:utility.obj
 0001:00000728       ___scrt_initialize_onexit_tables 10001728 f   MSVCRT:utility.obj
 0001:000007af       ___scrt_is_nonwritable_in_current_image 100017af f   MSVCRT:utility.obj
 0001:00000843       ___scrt_release_startup_lock 10001843 f   MSVCRT:utility.obj
 0001:00000860       ___scrt_uninitialize_crt   10001860 f   MSVCRT:utility.obj
 0001:00000888       ___scrt_get_dyn_tls_init_callback 10001888 f   MSVCRT:dyn_tls_init.obj
 0001:0000088e       ___scrt_fastfail           1000188e f   MSVCRT:utility_desktop.obj
 0001:000009a8       __crt_debugger_hook        100019a8 f   MSVCRT:utility_desktop.obj
 0001:000009b0       __RTC_Initialize           100019b0 f   MSVCRT:initsect.obj
 0001:000009dc       __RTC_Terminate            100019dc f   MSVCRT:initsect.obj
 0001:00000a10       __SEH_prolog4              10001a10 f   MSVCRT:sehprolg4.obj
 0001:00000a54       __SEH_epilog4              10001a54 f   MSVCRT:sehprolg4.obj
 0001:00000a68       __except_handler4          10001a68 f   MSVCRT:chandler4gs.obj
 0001:00000a97       @_guard_check_icall_nop@4  10001a97 f i MSVCRT:guard_support.obj
 0001:00000a9a       ___isa_available_init      10001a9a f   MSVCRT:cpu_disp.obj
 0001:00000c6a       __get_startup_argv_mode    10001c6a f   MSVCRT:argv_mode.obj
 0001:00000c6e       ___scrt_is_ucrt_dll_in_use 10001c6e f   MSVCRT:ucrt_detection.obj
 0001:00000c7a       @__security_check_cookie@4 10001c7a f   MSVCRT:secchk.obj
 0001:00000c8b       ___raise_securityfailure   10001c8b f   MSVCRT:gs_report.obj
 0001:00000cb3       ___report_gsfailure        10001cb3 f   MSVCRT:gs_report.obj
 0001:00000dac       _IsProcessorFeaturePresent@4 10001dac f   kernel32:KERNEL32.dll
 0001:00000db2       ___std_exception_copy      10001db2 f   vcruntime:VCRUNTIME140.dll
 0001:00000db8       ___std_exception_destroy   10001db8 f   vcruntime:VCRUNTIME140.dll
 0001:00000dbe       __CxxThrowException@8      10001dbe f   vcruntime:VCRUNTIME140.dll
 0001:00000dc4       ___std_type_info_destroy_list 10001dc4 f   vcruntime:VCRUNTIME140.dll
 0001:00000dca       _memset                    10001dca f   vcruntime:VCRUNTIME140.dll
 0001:00000dd0       __except_handler4_common   10001dd0 f   vcruntime:VCRUNTIME140.dll
 0001:00000dd6       __initterm                 10001dd6 f   ucrt:api-ms-win-crt-runtime-l1-1-0.dll
 0001:00000ddc       __initterm_e               10001ddc f   ucrt:api-ms-win-crt-runtime-l1-1-0.dll
 0001:00000de2       _free                      10001de2 f   ucrt:api-ms-win-crt-heap-l1-1-0.dll
 0001:00000de8       __seh_filter_dll           10001de8 f   ucrt:api-ms-win-crt-runtime-l1-1-0.dll
 0001:00000dee       __configure_narrow_argv    10001dee f   ucrt:api-ms-win-crt-runtime-l1-1-0.dll
 0001:00000df4       __initialize_narrow_environment 10001df4 f   ucrt:api-ms-win-crt-runtime-l1-1-0.dll
 0001:00000dfa       __initialize_onexit_table  10001dfa f   ucrt:api-ms-win-crt-runtime-l1-1-0.dll
 0001:00000e00       __execute_onexit_table     10001e00 f   ucrt:api-ms-win-crt-runtime-l1-1-0.dll
 0001:00000e06       __cexit                    10001e06 f   ucrt:api-ms-win-crt-runtime-l1-1-0.dll
 0001:00000e0c       ___acrt_uninitialize       10001e0c f   MSVCRT:ucrt_stubs.obj
 0001:00000e0c       ___vcrt_uninitialize       10001e0c f   MSVCRT:ucrt_stubs.obj
 0001:00000e0c       ___scrt_stub_for_acrt_uninitialize_critical 10001e0c f   MSVCRT:ucrt_stubs.obj
 0001:00000e0c       ___scrt_stub_for_acrt_uninitialize 10001e0c f   MSVCRT:ucrt_stubs.obj
 0001:00000e0c       ___acrt_thread_detach      10001e0c f   MSVCRT:ucrt_stubs.obj
 0001:00000e0c       ___scrt_stub_for_acrt_initialize 10001e0c f   MSVCRT:ucrt_stubs.obj
 0001:00000e0c       ___vcrt_initialize         10001e0c f   MSVCRT:ucrt_stubs.obj
 0001:00000e0c       ___vcrt_thread_detach      10001e0c f   MSVCRT:ucrt_stubs.obj
 0001:00000e0c       ___vcrt_uninitialize_critical 10001e0c f   MSVCRT:ucrt_stubs.obj
 0001:00000e0c       ___vcrt_thread_attach      10001e0c f   MSVCRT:ucrt_stubs.obj
 0001:00000e0c       ___scrt_stub_for_acrt_thread_attach 10001e0c f   MSVCRT:ucrt_stubs.obj
 0001:00000e0c       ___acrt_initialize         10001e0c f   MSVCRT:ucrt_stubs.obj
 0001:00000e0c       ___acrt_thread_attach      10001e0c f   MSVCRT:ucrt_stubs.obj
 0001:00000e0c       ___acrt_uninitialize_critical 10001e0c f   MSVCRT:ucrt_stubs.obj
 0001:00000e0c       ___scrt_stub_for_acrt_thread_detach 10001e0c f   MSVCRT:ucrt_stubs.obj
 0001:00000e0f       ___scrt_stub_for_is_c_termination_complete 10001e0f f   MSVCRT:ucrt_stubs.obj
 0001:00000e0f       __is_c_termination_complete 10001e0f f   MSVCRT:ucrt_stubs.obj
 0001:00000e12       __filter_x86_sse2_floating_point_exception_default 10001e12 f   MSVCRT:x86_exception_filter.obj
 0001:00000e12       __filter_x86_sse2_floating_point_exception 10001e12 f   MSVCRT:x86_exception_filter.obj
 0002:00000000       __imp__GetCurrentProcess@0 10002000     kernel32:KERNEL32.dll
 0002:00000004       __imp__GetModuleHandleA@4  10002004     kernel32:KERNEL32.dll
 0002:00000008       __imp__GetProcAddress@8    10002008     kernel32:KERNEL32.dll
 0002:0000000c       __imp__QueryPerformanceCounter@4 1000200c     kernel32:KERNEL32.dll
 0002:00000010       __imp__GetCurrentProcessId@0 10002010     kernel32:KERNEL32.dll
 0002:00000014       __imp__GetCurrentThreadId@0 10002014     kernel32:KERNEL32.dll
 0002:00000018       __imp__GetSystemTimeAsFileTime@4 10002018     kernel32:KERNEL32.dll
 0002:0000001c       __imp__InitializeSListHead@4 1000201c     kernel32:KERNEL32.dll
 0002:00000020       __imp__IsDebuggerPresent@0 10002020     kernel32:KERNEL32.dll
 0002:00000024       __imp__UnhandledExceptionFilter@4 10002024     kernel32:KERNEL32.dll
 0002:00000028       __imp__SetUnhandledExceptionFilter@4 10002028     kernel32:KERNEL32.dll
 0002:0000002c       __imp__IsProcessorFeaturePresent@4 1000202c     kernel32:KERNEL32.dll
 0002:00000030       __imp__TerminateProcess@8  10002030     kernel32:KERNEL32.dll
 0002:00000034       \177KERNEL32_NULL_THUNK_DATA 10002034     kernel32:KERNEL32.dll
 0002:00000038       __imp____std_exception_copy 10002038     vcruntime:VCRUNTIME140.dll
 0002:0000003c       __imp____std_exception_destroy 1000203c     vcruntime:VCRUNTIME140.dll
 0002:00000040       __imp___CxxThrowException@8 10002040     vcruntime:VCRUNTIME140.dll
 0002:00000044       __imp____std_type_info_destroy_list 10002044     vcruntime:VCRUNTIME140.dll
 0002:00000048       __imp__memset              10002048     vcruntime:VCRUNTIME140.dll
 0002:0000004c       __imp___except_handler4_common 1000204c     vcruntime:VCRUNTIME140.dll
 0002:00000050       \177VCRUNTIME140_NULL_THUNK_DATA 10002050     vcruntime:VCRUNTIME140.dll
 0002:00000054       __imp__free                10002054     ucrt:api-ms-win-crt-heap-l1-1-0.dll
 0002:00000058       \177api-ms-win-crt-heap-l1-1-0_NULL_THUNK_DATA 10002058     ucrt:api-ms-win-crt-heap-l1-1-0.dll
 0002:0000005c       __imp___initterm_e         1000205c     ucrt:api-ms-win-crt-runtime-l1-1-0.dll
 0002:00000060       __imp___seh_filter_dll     10002060     ucrt:api-ms-win-crt-runtime-l1-1-0.dll
 0002:00000064       __imp___configure_narrow_argv 10002064     ucrt:api-ms-win-crt-runtime-l1-1-0.dll
 0002:00000068       __imp___initialize_narrow_environment 10002068     ucrt:api-ms-win-crt-runtime-l1-1-0.dll
 0002:0000006c       __imp___initialize_onexit_table 1000206c     ucrt:api-ms-win-crt-runtime-l1-1-0.dll
 0002:00000070       __imp___initterm           10002070     ucrt:api-ms-win-crt-runtime-l1-1-0.dll
 0002:00000074       __imp___execute_onexit_table 10002074     ucrt:api-ms-win-crt-runtime-l1-1-0.dll
 0002:00000078       __imp___cexit              10002078     ucrt:api-ms-win-crt-runtime-l1-1-0.dll
 0002:0000007c       \177api-ms-win-crt-runtime-l1-1-0_NULL_THUNK_DATA 1000207c     ucrt:api-ms-win-crt-runtime-l1-1-0.dll
 0002:00000080       ___guard_check_icall_fptr  10002080     MSVCRT:guard_support.obj
 0002:00000084       ___xc_a                    10002084     MSVCRT:initializers.obj
 0002:00000088       ___xc_z                    10002088     MSVCRT:initializers.obj
 0002:0000008c       ___xi_a                    1000208c     MSVCRT:initializers.obj
 0002:00000090       ___xi_z                    10002090     MSVCRT:initializers.obj
 0002:00000094       ___xp_a                    10002094     MSVCRT:initializers.obj
 0002:00000098       ___xp_z                    10002098     MSVCRT:initializers.obj
 0002:0000009c       ___xt_a                    1000209c     MSVCRT:initializers.obj
 0002:000000a0       ___xt_z                    100020a0     MSVCRT:initializers.obj
 0002:000000ac       ??_7exception@std@@6B@     100020ac     AccessBridgeSysInfo.obj
 0002:000000b4       ??_C@_0BC@EOODALEL@Unknown?5exception@ 100020b4     AccessBridgeSysInfo.obj
 0002:000000cc       ??_7runtime_error@std@@6B@ 100020cc     AccessBridgeSysInfo.obj
 0002:000000d4       ??_C@_0P@LKABJJMO@IsWow64Process@ 100020d4     AccessBridgeSysInfo.obj
 0002:000000e4       ??_C@_08PNLNEKOB@kernel32@ 100020e4     AccessBridgeSysInfo.obj
 0002:000000f0       ??_C@_0BK@GDPMFCOH@fnIsWow64Process?$CI?$CJ?5failed@ 100020f0     AccessBridgeSysInfo.obj
 0002:00000110       ??_7type_info@@6B@         10002110     MSVCRT:std_type_info_static.obj
 0002:00000114       __pRawDllMain              10002114     MSVCRT:dll_dllmain.obj
 0002:00000114       __pDefaultRawDllMain       10002114     MSVCRT:dll_dllmain.obj
 0002:00000190       __load_config_used         10002190     MSVCRT:loadcfg.obj
 0002:00000248       ??_R4exception@std@@6B@    10002248     AccessBridgeSysInfo.obj
 0002:0000025c       ??_R3exception@std@@8      1000225c     AccessBridgeSysInfo.obj
 0002:0000026c       ??_R2exception@std@@8      1000226c     AccessBridgeSysInfo.obj
 0002:00000274       ??_R1A@?0A@EA@exception@std@@8 10002274     AccessBridgeSysInfo.obj
 0002:00000290       ??_R4runtime_error@std@@6B@ 10002290     AccessBridgeSysInfo.obj
 0002:000002a4       ??_R3runtime_error@std@@8  100022a4     AccessBridgeSysInfo.obj
 0002:000002b4       ??_R2runtime_error@std@@8  100022b4     AccessBridgeSysInfo.obj
 0002:000002c0       ??_R1A@?0A@EA@runtime_error@std@@8 100022c0     AccessBridgeSysInfo.obj
 0002:000002dc       ??_R4type_info@@6B@        100022dc     MSVCRT:std_type_info_static.obj
 0002:000002f0       ??_R3type_info@@8          100022f0     MSVCRT:std_type_info_static.obj
 0002:00000300       ??_R2type_info@@8          10002300     MSVCRT:std_type_info_static.obj
 0002:00000308       ??_R1A@?0A@EA@type_info@@8 10002308     MSVCRT:std_type_info_static.obj
 0002:00000324       ___safe_se_handler_table   10002324     <linker-defined>
 0002:000005d4       ___rtc_iaa                 100025d4     MSVCRT:initsect.obj
 0002:000005d8       ___rtc_izz                 100025d8     MSVCRT:initsect.obj
 0002:000005dc       ___rtc_taa                 100025dc     MSVCRT:initsect.obj
 0002:000005e0       ___rtc_tzz                 100025e0     MSVCRT:initsect.obj
 0002:000005e8       __CT??_R0?AVexception@std@@@8??0exception@std@@QAE@ABV01@@Z12 100025e8     AccessBridgeSysInfo.obj
 0002:00000604       __CT??_R0?AVruntime_error@std@@@8??0runtime_error@std@@QAE@ABV01@@Z12 10002604     AccessBridgeSysInfo.obj
 0002:00000620       __TI2?AVruntime_error@std@@ 10002620     AccessBridgeSysInfo.obj
 0002:00000630       __CTA2?AVruntime_error@std@@ 10002630     AccessBridgeSysInfo.obj
 0002:00000754       __IMPORT_DESCRIPTOR_KERNEL32 10002754     kernel32:KERNEL32.dll
 0002:00000768       __IMPORT_DESCRIPTOR_VCRUNTIME140 10002768     vcruntime:VCRUNTIME140.dll
 0002:0000077c       __IMPORT_DESCRIPTOR_api-ms-win-crt-runtime-l1-1-0 1000277c     ucrt:api-ms-win-crt-runtime-l1-1-0.dll
 0002:00000790       __IMPORT_DESCRIPTOR_api-ms-win-crt-heap-l1-1-0 10002790     ucrt:api-ms-win-crt-heap-l1-1-0.dll
 0002:000007a4       __NULL_IMPORT_DESCRIPTOR   100027a4     kernel32:KERNEL32.dll
 0003:00000000       ___scrt_native_dllmain_reason 10003000     MSVCRT:utility.obj
 0003:00000010       ___security_cookie_complement 10003010     MSVCRT:gs_cookie.obj
 0003:00000014       ___security_cookie         10003014     MSVCRT:gs_cookie.obj
 0003:00000018       ___isa_enabled             10003018     MSVCRT:cpu_disp.obj
 0003:0000001c       ___scrt_ucrt_dll_is_in_use 1000301c     MSVCRT:ucrt_stubs.obj
 0003:00000020       ??_R0?AVexception@std@@@8  10003020     AccessBridgeSysInfo.obj
 0003:0000003c       ??_R0?AVruntime_error@std@@@8 1000303c     AccessBridgeSysInfo.obj
 0003:0000005c       ??_R0?AVtype_info@@@8      1000305c     MSVCRT:std_type_info_static.obj
 0003:00000080       ?__type_info_root_node@@3U__type_info_node@@A 10003080     MSVCRT:tncleanup.obj
 0003:00000088       ?_OptionsStorage@?1??__local_stdio_printf_options@@9@4_KA 10003088     MSVCRT:default_local_stdio_options.obj
 0003:00000090       ?_OptionsStorage@?1??__local_stdio_scanf_options@@9@4_KA 10003090     MSVCRT:default_local_stdio_options.obj
 0003:00000098       ___scrt_current_native_startup_state 10003098     MSVCRT:utility.obj
 0003:0000009c       ___scrt_native_startup_lock 1000309c     MSVCRT:utility.obj
 0003:000000bc       ___scrt_debugger_hook_flag 100030bc     MSVCRT:utility_desktop.obj
 0003:000000c0       ___isa_available           100030c0     MSVCRT:cpu_disp.obj
 0003:000000c4       ___favor                   100030c4     MSVCRT:cpu_disp.obj
 0003:000003e4       ___dyn_tls_init_callback   100033e4     <common>

 entry point at        0001:000004af

 Static symbols

 0000:ffffa000       .debug$S                   10000000     jabsysinfo.exp
 0000:ffffa000       .debug$S                   10000000     vcruntime:VCRUNTIME140.dll
 0000:ffffa000       .debug$S                   10000000     vcruntime:VCRUNTIME140.dll
 0000:ffffa000       .debug$S                   10000000     vcruntime:VCRUNTIME140.dll
 0000:ffffa000       .debug$S                   10000000     vcruntime:VCRUNTIME140.dll
 0000:ffffa000       .debug$S                   10000000     vcruntime:VCRUNTIME140.dll
 0000:ffffa000       .debug$S                   10000000     vcruntime:VCRUNTIME140.dll
 0000:ffffa000       .debug$S                   10000000     vcruntime:VCRUNTIME140.dll
 0000:ffffa000       .debug$S                   10000000     vcruntime:VCRUNTIME140.dll
 0000:ffffa000       .debug$S                   10000000     ucrt:api-ms-win-crt-heap-l1-1-0.dll
 0000:ffffa000       .debug$S                   10000000     ucrt:api-ms-win-crt-runtime-l1-1-0.dll
 0000:ffffa000       .debug$S                   10000000     ucrt:api-ms-win-crt-runtime-l1-1-0.dll
 0000:ffffa000       .debug$S                   10000000     ucrt:api-ms-win-crt-runtime-l1-1-0.dll
 0000:ffffa000       .debug$S                   10000000     ucrt:api-ms-win-crt-runtime-l1-1-0.dll
 0000:ffffa000       .debug$S                   10000000     ucrt:api-ms-win-crt-runtime-l1-1-0.dll
 0000:ffffa000       .debug$S                   10000000     ucrt:api-ms-win-crt-runtime-l1-1-0.dll
 0000:ffffa000       .debug$S                   10000000     ucrt:api-ms-win-crt-runtime-l1-1-0.dll
 0000:ffffa000       .debug$S                   10000000     ucrt:api-ms-win-crt-runtime-l1-1-0.dll
 0000:ffffa000       .debug$S                   10000000     ucrt:api-ms-win-crt-runtime-l1-1-0.dll
 0000:ffffa000       .debug$S                   10000000     ucrt:api-ms-win-crt-runtime-l1-1-0.dll
 0000:ffffa000       .debug$S                   10000000     ucrt:api-ms-win-crt-runtime-l1-1-0.dll
 0000:ffffa000       .debug$S                   10000000     ucrt:api-ms-win-crt-runtime-l1-1-0.dll
 0000:ffffa000       .debug$S                   10000000     kernel32:KERNEL32.dll
 0000:ffffa000       .debug$S                   10000000     kernel32:KERNEL32.dll
 0000:ffffa000       .debug$S                   10000000     kernel32:KERNEL32.dll
 0000:ffffa000       .debug$S                   10000000     kernel32:KERNEL32.dll
 0000:ffffa000       .debug$S                   10000000     kernel32:KERNEL32.dll
 0000:ffffa000       .debug$S                   10000000     kernel32:KERNEL32.dll
 0000:ffffa000       .debug$S                   10000000     kernel32:KERNEL32.dll
 0000:ffffa000       .debug$S                   10000000     kernel32:KERNEL32.dll
 0000:ffffa000       .debug$S                   10000000     kernel32:KERNEL32.dll
 0000:ffffa000       .debug$S                   10000000     kernel32:KERNEL32.dll
 0000:ffffa000       .debug$S                   10000000     kernel32:KERNEL32.dll
 0000:ffffa000       .debug$S                   10000000     kernel32:KERNEL32.dll
 0000:ffffa000       .debug$S                   10000000     kernel32:KERNEL32.dll
 0000:ffffa000       .debug$S                   10000000     kernel32:KERNEL32.dll
 0000:ffffa000       .debug$S                   10000000     kernel32:KERNEL32.dll
 0001:0000016f       ?dllmain_crt_dispatch@@YGHQAUHINSTANCE__@@KQAX@Z 1000116f f   MSVCRT:dll_dllmain.obj
 0001:000001c2       ?dllmain_crt_process_attach@@YAHQAUHINSTANCE__@@QAX@Z 100011c2 f   MSVCRT:dll_dllmain.obj
 0001:000002c9       ?dllmain_crt_process_detach@@YAH_N@Z 100012c9 f   MSVCRT:dll_dllmain.obj
 0001:00000379       ?dllmain_dispatch@@YAHQAUHINSTANCE__@@KQAX@Z 10001379 f   MSVCRT:dll_dllmain.obj
 0001:00000484       ?dllmain_raw@@YGHQAUHINSTANCE__@@KQAX@Z 10001484 f   MSVCRT:dll_dllmain.obj
 0001:000004d7       ___get_entropy             100014d7 f   MSVCRT:gs_support.obj
 0001:000005b0       ?find_pe_section@@YAPAU_IMAGE_SECTION_HEADER@@QAEI@Z 100015b0 f   MSVCRT:utility.obj
 0001:00000a10       $$000000                   10001a10     MSVCRT:sehprolg4.obj
 0002:00000118       _GS_ExceptionPointers      10002118     MSVCRT:gs_report.obj
 0002:00000640       __sehtable$?dllmain_crt_process_attach@@YAHQAUHINSTANCE__@@QAX@Z 10002640     MSVCRT:dll_dllmain.obj
 0002:00000660       __sehtable$?dllmain_crt_process_detach@@YAH_N@Z 10002660     MSVCRT:dll_dllmain.obj
 0002:00000688       __sehtable$?dllmain_dispatch@@YAHQAUHINSTANCE__@@KQAX@Z 10002688     MSVCRT:dll_dllmain.obj
 0002:000006a8       __sehtable$___scrt_is_nonwritable_in_current_image 100026a8     MSVCRT:utility.obj
 0002:000006d0       .edata                     100026d0     jabsysinfo.exp
 0002:000006f8       rgpv                       100026f8     jabsysinfo.exp
 0002:000006fc       rgszName                   100026fc     jabsysinfo.exp
 0002:00000700       rgwOrd                     10002700     jabsysinfo.exp
 0002:00000702       szName                     10002702     jabsysinfo.exp
 0002:00000711       $N00001                    10002711     jabsysinfo.exp
 0002:00000966       .idata$6                   10002966     kernel32:KERNEL32.dll
 0002:00000a00       .idata$6                   10002a00     vcruntime:VCRUNTIME140.dll
 0002:00000ac0       .idata$6                   10002ac0     ucrt:api-ms-win-crt-runtime-l1-1-0.dll
 0002:00000ae2       .idata$6                   10002ae2     ucrt:api-ms-win-crt-heap-l1-1-0.dll
 0003:00000078       ?__proc_attached@@3HA      10003078     MSVCRT:dll_dllmain.obj
 0003:000000a0       ?is_initialized_as_dll@@3_NA 100030a0     MSVCRT:utility.obj
 0003:000000a1       ?module_local_atexit_table_initialized@@3_NA 100030a1     MSVCRT:utility.obj
 0003:000000a4       ?module_local_atexit_table@@3U_onexit_table_t@@A 100030a4     MSVCRT:utility.obj
 0003:000000b0       ?module_local_at_quick_exit_table@@3U_onexit_table_t@@A 100030b0     MSVCRT:utility.obj
 0003:000000c8       _GS_ExceptionRecord        100030c8     MSVCRT:gs_report.obj
 0003:00000118       _GS_ContextRecord          10003118     MSVCRT:gs_report.obj
 0004:00000120       $R000000                   10004120     jabsysinfo.dll.res
 0004:00000490       $R000370                   10004490     jabsysinfo.dll.res
 0004:000006a8       $R000588                   100046a8     jabsysinfo.dll.res
